:020000040801F1
:10000000000002202D30010805170108091701081A
:100010000D1701081117010815170108000000004D
:100020000000000000000000000000001917010897
:100030001D170108000000002117010825170108FD
:100040007D3001087D3001087D3001087D300108D8
:100050007D3001087D3001087D3001087D300108C8
:100060007D3001087D3001087D3001087D300108B8
:100070007D3001087D3001087D3001087D300108A8
:100080007D3001087D3001087D3001087D30010898
:100090007D3001087D3001087D3001087D30010888
:1000A0007D3001087D3001087D3001087D30010878
:1000B0007D3001087D3001087D3001087D30010868
:1000C0007D3001087D3001087D3001087D30010858
:1000D0007D30010835170108411701087D300108FE
:1000E0007D3001087D3001087D3001087D30010838
:1000F0007D3001087D3001087D3001087D30010828
:100100007D3001087D3001087D3001087D30010817
:100110004D1701087D3001087D3001087D30010850
:100120007D3001087D3001087D3001087D300108F7
:100130007D3001087D3001087D3001087D300108E7
:100140007D3001087D3001087D3001087D300108D7
:100150007D3001087D3001087D3001087D300108C7
:100160007D3001087D3001087D3001087D300108B7
:100170007D3001087D3001087D300108000000005D
:080180007D3001087D3001080B
:10018800044B05481B1A062B02D9044B03B1184728
:10019800704700BF3B00002038000020000000002E
:1001A80005490648091A891001EBD171491002D096
:1001B800034B03B11847704738000020380000206F
:1001C8000000000010B5064C237843B9FFF7D8FFAC
:1001D800044B13B10448AFF300800123237010BD12
:1001E80038000020000000008030010808B5084BE6
:1001F8001BB108490848AFF300800848036813B9E1
:10020800BDE80840CCE7064B002BF9D09847F7E744
:10021800000000003C000020803001083800002069
:100228000000000070B50F4E0F4D761BB61018BFBA
:10023800002405D0013455F8043B9847A642F9D16B
:100248000A4E0B4D761B02F017FFB61018BF00249C
:1002580006D0013455F8043B9847A642F9D170BD41
:1002680070BD00BFA8300108A8300108AC300108F3
:10027800A830010870B4860746D0541E002A41D021
:10028800CAB2034602E014F1FF343BD303F8012B52
:100298009D07F8D1032C2ED9CDB245EA05250F2CA0
:1002A80045EA054519D903F110022646103E0F2EDE
:1002B80042F8105C42F80C5C42F8085C42F8045CB6
:1002C80002F11002F2D8A4F1100222F00F0204F099
:1002D8000F041032032C13440DD91E462246043A4B
:1002E800032A46F8045BFAD8221F22F003020432DC
:1002F800134404F003042CB1C9B21C4403F8011BD5
:100308009C42FBD170BC704714460346C2E700BF4D
:1003180081F0004102E000BF83F0004330B54FEAAE
:1003280041044FEA430594EA050F08BF90EA020F1B
:100338001FBF54EA000C55EA020C7FEA645C7FEAAE
:10034800655C00F0E2804FEA5454D4EB5555B8BFD1
:100358006D420CDD2C4480EA020281EA030382EA42
:10036800000083EA010180EA020281EA0303362DD4
:1003780088BF30BD11F0004F4FEA01314FF4801CA7
:100388004CEA113102D0404261EB410113F0004FB9
:100398004FEA03334CEA133302D0524263EB430370
:1003A80094EA050F00F0A780A4F10104D5F1200E0E
:1003B8000DDB02FA0EFC22FA05F2801841F1000169
:1003C80003FA0EF2801843FA05F359410EE0A5F13D
:1003D80020050EF1200E012A03FA0EFC28BF4CF06E
:1003E800020C43FA05F3C01851EBE37101F0004524
:1003F80007D54FF0000EDCF1000C7EEB00006EEB31
:100408000101B1F5801F1BD3B1F5001F0CD34908BA
:100418005FEA30004FEA3C0C04F101044FEA445211
:1004280012F5800F80F09A80BCF1004F08BF5FEA98
:10043800500C50F1000041EB045141EA050130BD78
:100448005FEA4C0C404141EB010111F4801FA4F11B
:100458000104E9D191F0000F04BF01460020B1FA70
:1004680081F308BF2033A3F10B03B3F120020CDAA8
:100478000C3208DD02F1140CC2F10C0201FA0CF086
:1004880021FA02F10CE002F11402D8BFC2F1200CEB
:1004980001FA02F120FA0CFCDCBF41EA0C019040A1
:1004A800E41AA2BF01EB0451294330BD6FEA0404EA
:1004B8001F3C1CDA0C340EDC04F11404C4F12002D5
:1004C80020FA04F001FA02F340EA030021FA04F3E7
:1004D80045EA030130BDC4F10C04C4F1200220FA3E
:1004E80002F001FA04F340EA0300294630BD21FA7C
:1004F80004F0294630BD94F0000F83F4801306BF42
:1005080081F480110134013D4EE77FEA645C18BF35
:100518007FEA655C29D094EA050F08BF90EA020FCC
:1005280005D054EA000C04BF1946104630BD91EAC4
:10053800030F1EBF0021002030BD5FEA545C05D1C7
:100548004000494128BF41F0004130BD14F5800406
:100558003CBF01F5801130BD01F0004545F0FE417A
:1005680041F470014FF0000030BD7FEA645C1ABFAF
:10057800194610467FEA655C1CBF0B46024650EAE6
:10058800013406BF52EA033591EA030F41F4002112
:1005980030BD00BF90F0000F04BF0021704730B598
:1005A8004FF4806404F132044FF000054FF000016D
:1005B80050E700BF90F0000F04BF0021704730B52E
:1005C8004FF4806404F1320410F0004548BF404203
:1005D8004FF000013EE700BF42004FEAE2014FEA58
:1005E80031014FEA02701FBF12F07F4393F07F4F33
:1005F80081F06051704792F0000F14BF93F07F4F65
:10060800704730B54FF4607401F0004521F00041A7
:1006180020E700BF50EA010208BF704730B54FF02D
:1006280000050AE050EA010208BF704730B511F032
:10063800004502D5404261EB41014FF4806404F16A
:1006480032045FEA915C3FF4DCAE4FF003025FEAEC
:10065800DC0C18BF03325FEADC0C18BF033202EB74
:10066800DC02C2F1200300FA03FC20FA02F001FACE
:1006780003FE40EA0E0021FA02F11444C1E600BF6D
:1006880070B54FF0FF0C4CF4E06C1CEA11541DBF20
:100698001CEA135594EA0C0F95EA0C0F00F0DEF8EB
:1006A8002C4481EA030621EA4C5123EA4C5350EAD0
:1006B800013518BF52EA033541F4801143F4801321
:1006C80038D0A0FB02CE4FF00005E1FB02E506F0B2
:1006D8000042E0FB03E54FF00006E1FB03569CF007
:1006E800000F18BF4EF0010EA4F1FF04B6F5007F0D
:1006F80064F5407404D25FEA4E0E6D4146EB06067F
:1007080042EAC62141EA55514FEAC52040EA5E5007
:100718004FEACE2EB4F1FD0C88BFBCF5E06F1ED8B1
:10072800BEF1004F08BF5FEA500E50F1000041EBE8
:10073800045170BD06F0004646EA010140EA020095
:1007480081EA0301B4EB5C04C2BFD4EB0C0541EAB7
:10075800045170BD41F480114FF0000E013C00F3CC
:10076800AB8014F1360FDEBF002001F0004170BDF0
:10077800C4F10004203C35DA0C341BDC04F1140409
:10078800C4F1200500FA05F320FA04F001FA05F295
:1007980040EA020001F0004221F0004110EBD37062
:1007A80021FA04F642EB06015EEA430E08BF20EA8E
:1007B800D37070BDC4F10C04C4F1200500FA04F331
:1007C80020FA05F001FA04F240EA020001F00041C3
:1007D80010EBD37041F100015EEA430E08BF20EA36
:1007E800D37070BDC4F1200500FA05F24EEA020E7E
:1007F80020FA04F301FA05F243EA020321FA04F0AD
:1008080001F0004121FA04F220EA020000EBD37063
:100818005EEA430E08BF20EAD37070BD94F0000F63
:100828000FD101F00046400041EB010111F4801F97
:1008380008BF013CF7D041EA060195F0000F18BF48
:10084800704703F00046520043EB030313F4801F84
:1008580008BF013DF7D043EA0603704794EA0C0F3E
:100868000CEA135518BF95EA0C0F0CD050EA410654
:1008780018BF52EA4306D1D181EA030101F00041D1
:100888004FF0000070BD50EA410606BF10461946F9
:1008980052EA430619D094EA0C0F02D150EA013605
:1008A80013D195EA0C0F05D152EA03361CBF104646
:1008B80019460AD181EA030101F0004141F0FE41E5
:1008C80041F470014FF0000070BD41F0FE4141F469
:1008D800780170BD70B54FF0FF0C4CF4E06C1CEA69
:1008E80011541DBF1CEA135594EA0C0F95EA0C0F1E
:1008F80000F0A7F8A4EB050481EA030E52EA0335D9
:100908004FEA013100F088804FEA03334FF08055F9
:1009180045EA131343EA12634FEA022245EA111526
:1009280045EA10654FEA00260EF000419D4208BFD7
:10093800964244F1FD0404F5407402D25B084FEA84
:100948003202B61A65EB03055B084FEA32024FF430
:1009580080104FF4002CB6EB020E75EB030E22BF8D
:10096800B61A754640EA0C005B084FEA3202B6EB4D
:10097800020E75EB030E22BFB61A754640EA5C00FC
:100988005B084FEA3202B6EB020E75EB030E22BF8C
:10099800B61A754640EA9C005B084FEA3202B6EB8D
:1009A800020E75EB030E22BFB61A754640EADC004C
:1009B80055EA060E18D04FEA051545EA16754FEAAE
:1009C80006164FEAC30343EA52734FEAC2025FEACC
:1009D8001C1CC0D111F4801F0BD141EA00014FF05B
:1009E80000004FF0004CB6E711F4801F04BF01432C
:1009F8000020B4F1FD0C88BFBCF5E06F3FF6AFAE48
:100A0800B5EB030C04BFB6EB020C5FEA500C50F1D7
:100A1800000041EB045170BD0EF0004E4EEA11315A
:100A280014EB5C04C2BFD4EB0C0541EA045170BD61
:100A380041F480114FF0000E013C90E645EA060EA5
:100A48008DE60CEA135594EA0C0F08BF95EA0C0FD3
:100A58003FF43BAF94EA0C0F0AD150EA01347FF41B
:100A680034AF95EA0C0F7FF425AF104619462CE7F2
:100A780095EA0C0F06D152EA03353FF4FDAE104655
:100A8800194622E750EA410618BF52EA43067FF4A6
:100A9800C5AE50EA41047FF40DAF52EA43057FF436
:100AA800EBAE12E74FF0FF3C06E000BF4FF0010C41
:100AB80002E000BF4FF0010C4DF804CD4FEA410CA5
:100AC8007FEA6C5C4FEA430C18BF7FEA6C5C1BD072
:100AD80001B050EA410C0CBF52EA430C91EA030FF3
:100AE80002BF90EA020F0020704710F1000F91EA50
:100AF800030F58BF994208BF90422CBFD8176FEA1E
:100B0800E37040F0010070474FEA410C7FEA6C5CEB
:100B180002D150EA013C07D14FEA430C7FEA6C5CF2
:100B2800D6D152EA033CD3D05DF8040B704700BF1E
:100B38008446104662468C461946634600E000BF6C
:100B480001B5FFF7B7FF002848BF10F1000F01BD3E
:100B58004DF808EDFFF7F4FF0CBF012000205DF809
:100B680008FB00BF4DF808EDFFF7EAFF34BF01208E
:100B780000205DF808FB00BF4DF808EDFFF7E0FF27
:100B880094BF012000205DF808FB00BF4DF808ED78
:100B9800FFF7CEFF94BF012000205DF808FB00BFDF
:100BA8004DF808EDFFF7C4FF34BF012000205DF8C1
:100BB80008FB00BF4FEA410212F5001215D211D509
:100BC8006FF47873B3EB625212D94FEAC12343F042
:100BD800004343EA505311F0004F23FA02F018BFC4
:100BE800404270474FF00000704750EA013005D18D
:100BF80011F0004008BF6FF0004070474FF0000050
:100C0800704700BF4A0011D212F5001211D20DD55B
:100C18006FF47873B3EB62520ED44FEAC12343F0FA
:100C2800004343EA505323FA02F070474FF00000A4
:100C3800704750EA013002D14FF0FF3070474FF053
:100C480000007047F0B595B008A830220021FFF7E2
:100C580011FB00241D4A01940494039405940694FE
:100C68000794116C1A4B41F080511164126C02F018
:100C780080520192019A02941A6842F480421A60E2
:100C88001B680F9403F48043029301230225082173
:100C980048220B9308A8032310261091119213934E
:100CA800029F08950E9512950C9601F0C9FC0F222B
:100CB8004FF4805303A8294604950594079403929A
:100CC800069301F0B3FE15B0F0BD00BF0038024036
:100CD800007000402DE9F043DFF86880174C184F8A
:100CE80085B0ED25012602952946334600944046F5
:100CF8000196FA2200F0DCFF02958DE85000334699
:100D0800387029464046FB2294F8009000F0D0FF46
:100D180002953346387029468DE8500025784046BC
:100D2800FC2200F0C5FF2D012378387045EA09350B
:100D380045EA131005B0BDE8F08300BF6800002045
:100D48006C000020A40000202DE9F043DFF8688043
:100D5800174C184F85B0ED250126029529463346D4
:100D6800009440460196F72200F0A2FF02958DE814
:100D780050003346387029464046F82294F80090CF
:100D880000F096FF02953346387029468DE85000EA
:100D980025784046F92200F08BFF2D012378387022
:100DA80045EA093545EA131005B0BDE8F08300BFF0
:100DB800680000206C000020A40000200000000053
:100DC8002DE9F047FFF786FFC34C2060FFF7BCFF13
:100DD800C24B8246C3F800A02068FFF7DBFBC04B7C
:100DE800064618880F46FFF7D5FB002204460D4635
:100DF800BC4B30463946FFF743FC00228046894603
:100E0800B94B20462946FFF73BFC02460B464046B5
:100E18004946FFF781FA002280468946B34B30469F
:100E28003946FFF72DFC002206460F46B04B2046F8
:100E38002946FFF725FC02460B4630463946FFF7A0
:100E48006BFAAC4B044618880D46FFF7A3FB024625
:100E58000B4620462946FFF713FCA74B0446188883
:100E68000D46FFF797FB424606460F464B4640465F
:100E78004946FFF705FC02460B4630463946FFF760
:100E8800FFFB02460B4620462946FFF747FAFFF7C5
:100E980091FEFFF78FFB0022984BFFF7F1FB002232
:100EA800974BFFF739FA974B044618880D46FFF71A
:100EB80071FB224606460F462B4620462946FFF779
:100EC800DFFB02460B4630463946FFF7D9FB0022C6
:100ED8004FF07C53FFF7D4FB8B4B064618880F4620
:100EE800FFF758FB22462B46FFF7CAFB02460B4684
:100EF800FFF714FA32463B46FFF710FA0022834BFD
:100F0800FFF7BEFB824B064618880F46FFF742FBE9
:100F18000022804BFFF7B4FB32463B46FFF7FEF951
:100F28007D4B804618888946FFF734FB22462B46BE
:100F3800FFF7A6FB22462B46FFF7A2FB00224FF045
:100F48007B53FFF79DFB754B064618880F46FFF746
:100F580021FB22462B46FFF793FB02460B46304601
:100F68003946FFF7DBF900224FF07B53FFF788FB88
:100F780000224FF07C53FFF783FB0022684BFFF7FA
:100F8800CDF9684B04460D461888FFF703FB224647
:100F98002B46FFF775FB0022002304460D46FFF79A
:100FA800D7FD08B1002400255046FFF7F3FA0246A2
:100FB8000B4600205C49FFF7AFF9002206460F46B2
:100FC8005A4B40464946FFF75BFB02460B46304604
:100FD8003946FFF7A1F93CA3D3E90023FFF750FBFB
:100FE80022462B46FFF776FC514B524C524D064693
:100FF8000F461888FFF7CEFA32463B46FFF740FB0C
:1010080032463B46FFF73CFB00224FF07853FFF790
:1010180037FB4A4B804618888946FFF7BBFA3246A9
:101028003B46FFF72DFB00224FF07C53FFF728FBD0
:1010380002460B4640464946FFF770F9404B80464A
:1010480018888946FFF7A6FA02460B4640464946E5
:10105800FFF764F900223B4BFFF712FB02460B46F1
:1010680030463946FFF75AF919A3D3E90023064653
:101078000F46FFF72FFCFFF7C5FD39466070304675
:10108800FFF798FD3049024681FB0231D317C3EBC5
:10109800213342F2107707FB132385FB0312DD1778
:1010A800C5EB6215642606FB153621462748A57050
:1010B80001230722E67001F0EFF83846BDE8F04753
:1010C80001F07ABFAFF3008000000000006AB8406A
:1010D800000000000088C340600000205C00002081
:1010E800660000200000E03E0000203F0000103FA6
:1010F8000000503F6A0000209E0000200000E03FF2
:101108000040EF40A00000207E0000200000D03FFB
:101118007C0000200000F040820000207A000020BF
:101128000000F03F80000020000030410000303F08
:101138009C000020080000201F85EB51840000203F
:10114800640000200000B03FAD8BDB683801002050
:101158002DE9F043DFF85090124CDFF8508085B04D
:101168000126ED2507460246029529463346009496
:101178004846019600F09CFDBA1902953346294667
:1011880088F8000092B28DE850004846257800F0B3
:101198008FFD237888F8000045EA032000B205B0E7
:1011A800BDE8F08368000020A40000206C00002047
:1011B80080B5744B744A9A6084B001F0D5FEFFF78D
:1011C80041FD00F01FF900F0F3F900F0B9F900F063
:1011D800D3F90A2305226D496D486E4C01F05CF87D
:1011E8004FF47A7001F0E8FE0A2305226A4968483C
:1011F80001F052F821464FF4FA631422644801F0D2
:10120800A7F80A2314222146644801F045F8A37C74
:101218005A1E012A40F2AE80052B05D10A230B2263
:101228005F495E4801F038F85E4B5F485F4D604C9F
:10123800DFF8C881ED2710268DE8C800E0220123D9
:10124800EC2100F099FC5B4B02970196F422287080
:10125800EC2100935448012300F08EFC564B287073
:10126800F522EC218DE8C8004F48544F544E012315
:1012780000F082FC28708820FFF76AFF514B524D1E
:1012880018808A20FFF764FF504B18808C20FFF7E6
:101298005FFF4F4B18808E20FFF75AFF4D4B188089
:1012A8009020FFF755FF4C4B18809220FFF750FF16
:1012B8004A4B18809420FFF74BFF494B1880962023
:1012C800FFF746FF474B18809820FFF741FF464B32
:1012D80018809A20FFF73CFF444B18809C20FFF7AA
:1012E80037FF434B18809E20FFF732FF414B188091
:1012F800B3EE008AFFF764FDD4ED007AF4EEC87A05
:10130800F1EE10FAF6D5384600224FF4806101F06C
:101318008BFD384600224FF4807101F085FD304680
:1013280000224FF4004101F07FFD304600224FF4C7
:10133800005101F079FD304600224FF4006101F0C0
:1013480073FD404600224FF4004101F06DFD284630
:1013580000224FF4004101F067FD284600224FF4B7
:10136800005101F061FD00224FF40061284601F0B0
:101378005BFDBDE70A2307221F49084800F08CFFE0
:1013880052E700BF00ED00E000000108180000204F
:10139800780100208800002010000020380100207B
:1013A8002800002000000020A40000206C0000207D
:1013B80054000020040000205800002000000240D3
:1013C800000C024066000020001002406A00002065
:1013D8009E000020800000207A000020820000206B
:1013E8007C0000207E000020A00000206400002077
:1013F800840000209C0000202000002000040240FF
:10140800704700BF2DE9F0438BB00024464B009491
:101418001A6B464DDFF82091DFF82081444F454E86
:1014280042F001021A631A6B02F001020092009A5C
:1014380001941A6B42F010021A631A6B02F0100240
:101448000192019A02941A6B42F002021A631A6B13
:1014580002F002020292029A03941A6B42F0080206
:101468001A631A6B02F008020392039A04941A6B27
:1014780042F004021A631B6B03F00403049328462A
:1014880001224FF47841049B01F0CEFC484601222A
:101498004FF4404101F0C8FC404601224FF47C4122
:1014A80001F0C2FC384601224FF4007101F0BCFC87
:1014B800012230464FF47C5101F0B6FC284605A9BC
:1014C80001254FF47843059307940894069501F095
:1014D80095FB484605A94FF44043059306950794A4
:1014E800089401F08BFB404605A94FF47C43059313
:1014F80006950794089401F081FB384605A94FF436
:101508000073059306950794089401F077FB4FF450
:101518007C5305A93046069507940894059301F075
:101528006DFB0BB0BDE8F0830038024000100240AC
:10153800000802400000024000040240000C024083
:101548000B4B0C4A10B50C211A604FF4E134002201
:1015580018465C6059619A60DA601A619A61DA61CA
:1015680000F06AFE00B910BDBDE81040FFF748BFA3
:1015780038010020004C00400B4B0C4A10B50C21E0
:101588001A604FF4E134002218465C6059619A6091
:10159800DA601A619A61DA6100F04EFE00B910BD96
:1015A800BDE81040FFF72CBFF800002000100140F4
:1015B8000B4B0C4A10B50C211A604FF4164400224C
:1015C80018465C6059619A60DA601A619A61DA615A
:1015D80000F032FE00B910BDBDE81040FFF710BFA3
:1015E8007801002000440040F0B503683C4A93426B
:1015F80089B02BD03B4A93424DD03B4A934201D00D
:1016080009B0F0BD0024394B0294196C384841F4F4
:10161800003119641B6C03F400330293032207237F
:1016280003A9602702260125DDF808E00692079342
:1016380003970496059501F0E1FA224621462620F3
:1016480001F01AFC262001F04DFCD9E70024274BB5
:101658000094196C274841F4002119641B6C03F4A9
:10166800002300930322082303A94FF440670226AE
:101678000125DDF800E00692079303970496059587
:1016880001F0BCFA22462146342001F0F5FB342053
:1016980001F028FCB4E70024144B0194596C164857
:1016A80041F0100159645B6C03F0100301930322AD
:1016B800072303A9C02702260125DDF804E00692C6
:1016C800079303970496059501F098FA2246214658
:1016D800252001F0D1FB252001F004FC90E700BF94
:1016E800004C004000100140004400400038024017
:1016F800000C02400008024000040240704700BF8E
:10170800FEE700BFFEE700BFFEE700BFFEE700BF41
:10171800704700BF704700BF704700BF08B501F0B1
:101728003DFCBDE8084001F005BC00BF014800F0E1
:10173800B9BE00BFF8000020014800F0B3BE00BFEA
:1017480078010020014800F0ADBE00BF380100203C
:1017580008B5032001F07EFB002211466FF00B0054
:1017680001F08AFB002211466FF00A0001F084FBA9
:10177800002211466FF0090001F07EFB002211469D
:101788006FF0040001F078FB002211466FF00300AF
:1017980001F072FB002211466FF0010001F06CFBB2
:1017A800002211464FF0FF30BDE8084001F064BB4D
:1017B8002DE9F843074690469946C1F307468DB28E
:1017C8003C68012E1FD0A06935EA000314BF012030
:1017D800002000B3606943051FD4B8F1FF3FF0D083
:1017E800B8F1000F05D001F0E1FBA0EB090080453E
:1017F800E6D2002320223B6387F83C3087F83D205F
:101808000320BDE8F883626935EA020314BF0120AA
:1018180000200028DED1BDE8F883236800226FF499
:10182800806643F40073042520212360012066614B
:101838003D6487F83C203A6387F83D10BDE8F8839B
:101848002DE9F041804617461D46C1F307468CB284
:10185800D8F8001009E0886934EA00030CBF0120B9
:101868000020B8420BD16B1C0CD1012EF3D14B696F
:1018780034EA03030CBF01200020B842F3D0002053
:10188800BDE8F0812DB101F091FB069BC01A85429D
:10189800DED200232022C8F8303088F83C3088F89F
:1018A8003D20032088F83E30BDE8F081F8B50446B5
:1018B8000E4617462068436913F0040324D145698E
:1018C8006A050CD56FF480650421202245612164E6
:1018D8000120236384F83C3084F83D20F8BD731C54
:1018E800E9D026B101F062FBC01B8642E2D2236C2C
:1018F800002243F020032021236484F83C20226343
:10190800032084F83D10F8BD0020F8BD70B50546E9
:101918000C46164608E05169C90617D45CB101F0B7
:1019280045FB801B844206D32A68536913F04003A1
:10193800F1D0002070BD2B6C2022134300212B64B2
:1019480085F83C1085F83D20032070BD6FF010002D
:10195800202150612B6401202B6385F83C3085F8E9
:101968003D1070BDF8B504460E4617462068436919
:1019780013F0800324D145696A050CD56FF480659E
:1019880004212022456121640120236384F83C302E
:1019980084F83D20F8BD731CE9D026B101F006FBA0
:1019A800C01B8642E2D2236C002243F02003202190
:1019B800236484F83C202263032084F83D10F8BD9A
:1019C8000020F8BD2DE9F047056884B02C680D9E0D
:1019D80044F48074884691469A462C600C9B009685
:1019E80000224FF001110746FFF72AFF18B1032024
:1019F80004B0BDE8F0873A681E4908F0FE03136199
:101A0800384633460C9AFFF7D3FE20B13B6C042BC3
:101A1800EDD10120ECE73B6803905A6903929B697A
:101A2800039332460C99039B3846FFF79BFF88B90E
:101A3800BAF1010F18D039684FEA19230B61324601
:101A48000C993846FFF78EFF20B93A685FFA89F398
:101A58001361CDE73B6C042BC9D13A68136843F492
:101A6800007313600120C3E73B685FFA89F21A61CB
:101A7800BEE700BF020001002DE9F04704682568B1
:101A880045F48065256084B025680D9E45F4807511
:101A9800884691469A4625600C9B009600224FF096
:101AA80001110746FFF7CCFE18B1032004B0BDE8CA
:101AB800F0873B682F495FFA88F808F0FE021A6140
:101AC800384633460C9AFFF773FE20B13B6C042B63
:101AD800EBD10120EAE73B6803905A6903929B69BE
:101AE800039332460C99039B3846FFF73BFF60B9D6
:101AF800BAF1010F3B6811D15FFA89F21A613246D7
:101B08000C993846FFF72EFFB8B13B6C042BCCD1AB
:101B18003A68136843F400731360DAE74FEA19224E
:101B28001A610C9932463846FFF71CFF0028ECD1A1
:101B38003A685FFA89F31361E1E739680B6843F49F
:101B480080730B6002460C9B00964FF001113846DB
:101B5800FFF776FE0028A8D13A68064948F0010840
:101B6800C2F8108033460C9A3846FFF721FE002849
:101B7800ACD19BE7020001002DE9F047044682B092
:101B880098460E461746BDF82C9001F00FFA94F8C7
:101B98003D30202B03D0022002B0BDE8F087054677
:101BA80000901923012240492046FFF749FE0028EA
:101BB800F1D194F83C30012BEDD023681A6801214B
:101BC800D20784F83C1002D41A680A431A601A68CB
:101BD800364922F400621A604FF0000A212240239D
:101BE80084F83D2084F83E30C4F840A0A4F82A9038
:101BF800E162608D0A9B636231460C9E01950096F6
:101C0800434620853A462046FFF7DCFE002839D1B6
:101C1800238D0C992A462046B3B1FFF7A3FE00286E
:101C280037D1626A2168208D531C636213780B6177
:101C3800638D013B9BB263854E69431E9BB2760759
:101C48002385E6D5961C93B92A460C992046FFF7BA
:101C58002DFEF0B922681368202143F40073136045
:101C680084F83D1084F83C0084F83E0094E76662EE
:101C780053780B61628D831E013A9BB292B2238521
:101C88006285C6E7236C84F83CA0042B09D00320A6
:101C980082E7236C042BFAD12268136843F400739B
:101CA8001360012078E700BF020010000000FFFF6A
:101CB8002DE9F047044686B099460D469046BDF892
:101CC8003C7001F073F994F83D30202B04D00225C4
:101CD800284606B0BDE8F087064600901923012281
:101CE8007C492046FFF7ACFD0028F0D194F83C3041
:101CF800012BECD023681A680121D00784F83C1026
:101D080002D41A680A431A601A68734922F40062F6
:101D18001A604FF0000A2222402384F83D2084F8FC
:101D28003E30C4F840A06785E162608D0E9B636217
:101D38002946109D009501964B462085424620462F
:101D4800FFF79AFE054638B1236C84F83CA0042BB3
:101D580000F0A0800325BBE7238D9BB92368029080
:101D68005A6902929A690292029A1A6842F40072B7
:101D78001A600023202284F83D2084F83C3084F83F
:101D88003E30A5E7012B226800F08680022B00F088
:101D9800928005905169059192690592059ADFF83C
:101DA8003C81032B49D8012B65D0022F0096109B4C
:101DB8004FF000024146204619D0FFF741FD0028A8
:101DC800C8D12368626A196821F4806119601B69A7
:101DD800511C61621370638D218D0096013B9BB28B
:101DE80001396385109B2185024641462046FFF74D
:101DF80027FD0028AED12368616A1A6842F4007290
:101E08001A601B694A1C62620B70638D218D606ABF
:101E18002268013B9BB2638512694B1E411C2385D6
:101E280061620270238D628D013B013A9BB292B2CE
:101E380023856285002BB4D19BE732461099204652
:101E4800FFF764FD10BB636A2268591C126961625E
:101E58001A70628D2168238D013A92B262854A69AF
:101E6800013B9BB252072385E4D5636A0A69591C72
:101E780061621A70D6E7324610992046FFF746FD90
:101E880020B9636A2268591C1269F1E7236C202B78
:101E98003FF460AF01251BE7116821F480611160F0
:101EA800039051690391916903910399116841F471
:101EB8000071116073E7116821F480611160116885
:101EC80041F400611160049051690491926904928F
:101ED800049A64E7020010000000FFFF04000100FC
:101EE8002DE9F047046822698246C068DAF81C10B8
:101EF800DAF80830DAF81060DAF8145022F44052B0
:101F080002432261E268DAF81800334322F41642E9
:101F18002B4322F00C020B431343E360636923F461
:101F280040730343B1F5004F6361AB4B61D09C42F2
:101F380000F0018103F580639C4200F0FC8000F012
:101F48002DFEA64FDAF8043000EB800000EB80008D
:101F58009B00B0FBF3F3A7FB03235B091D0100F013
:101F68001DFEDAF8043000EB80009B0000EB8000D7
:101F7800B0FBF3F600F012FEDAF8042000EB800064
:101F8800930000EB8000B0FBF3F3A7FB03234FF0B3
:101F980064095B0909FB13631B013233A7FB0323A5
:101FA8005B0903F0F00600F0F9FDDAF8042000EB15
:101FB8008000930000EB8000B0FBF3F800F0EEFD2A
:101FC800DAF8043000EB80009B0000EB8000B0FBE7
:101FD800F3F0A7FB0030400909FB10831B013233E3
:101FE800A7FB0323C3F3431333432B44A360BDE888
:101FF800F0879C425DD003F580639C4259D000F085
:10200800CDFD764FDAF8043000EB800000EB80005D
:102018005B00B0FBF3F3A7FB03235B091E0100F091
:10202800BDFDDAF8043000EB80005B0000EB8000B7
:10203800B0FBF3F500F0B2FDDAF8042000EB800005
:10204800530000EB8000B0FBF3F3A7FB03235B090D
:102058004FF0640909FB1353DB003233A7FB03235A
:102068001B0903F4F87500F099FDDAF8042000EB79
:10207800800000EB80005300B0FBF3F800F08EFD09
:10208800DAF8043000EB800000EB80005B00B0FB66
:10209800F3F3A7FB03235B0909FB1383DB0032334C
:1020A800A7FB0323C3F3421333442B44A360BDE8C7
:1020B800F08700F08BFD494FDAF8043000EB800020
:1020C80000EB80005B00B0FBF3F3A7FB03235B0985
:1020D8001E0100F07BFDDAF8043000EB80005B00A5
:1020E80000EB8000B0FBF3F500F070FDDAF8042097
:1020F80000EB8000530000EB8000B0FBF3F3A7FB7C
:1021080003234FF064095B0909FB1353DB003233E7
:10211800A7FB03231B0903F4F87500F057FDDAF851
:10212800042000EB8000530000EB8000B0FBF3F8C4
:1021380000F04CFDA4E700F049FD284FDAF8043020
:1021480000EB800000EB80009B00B0FBF3F3A7FBE3
:1021580003235B091D0100F039FDDAF8043000EBB8
:1021680080009B0000EB8000B0FBF3F600F02EFD32
:10217800DAF8042000EB8000930000EB8000B0FB4D
:10218800F3F3A7FB03234FF064095B0909FB13630F
:102198001B013233A7FB03235B0903F0F00600F0B1
:1021A80015FDDAF8042000EB8000930000EB8000B6
:1021B800B0FBF3F800F00AFDDAF8043000EB800019
:1021C80000EB80009B00B0FBF3F3A7FB03235B0944
:1021D80009FB138302E700BF001001401F85EB5184
:1021E8002DE9F04107460E4690461D463C6801E041
:1021F8006B1C06D1206836EA0003F9D10020BDE83F
:10220800F08135B100F0D2FEA0EB08008542EDD296
:102218003C68E36823F4D073E3606369202223F009
:10222800010300216361032087F8392087F83810FB
:1022380087F83A20BDE8F08160B338B590F83930B6
:10224800044603F0FF0203B32268242384F83930DC
:10225800D36823F40053D3602046FFF741FE236878
:102268001A6922F490421A615A6922F02A025A61C4
:10227800DA680025202142F40052DA602846E56336
:1022880084F8391084F83A1038BD80F83820FFF700
:10229800ABF9D9E7012070472DE9F0430F4690F8D4
:1022A8003910202983B003D0022003B0BDE8F083A1
:1022B800002F3ED0002A3CD0984690F83830012BA9
:1022C8000446F1D0002001212123E06384F838106E
:1022D80084F83930019200F069FE019AA28481469F
:1022E800E28406E0FFF77CFF28BB23683A785A604F
:1022F8000137E58CADB243464A4680212046E5B118
:10230800E58CA668013DADB2B6F5805FE584E9D1FC
:1023180043464A4680212046FFF762FF58B93B886A
:1023280021682269C3F308034B60002AE0D1023711
:10233800DFE70120B9E70320B7E74021FFF750FFA7
:102348000028F8D1202384F8380084F83930ACE725
:102358002DE9F0430E4690F83A10202983B003D0B7
:10236800022003B0BDE8F08376B36AB3984690F8CC
:102378003830012B0446F3D0002001212223E063EA
:1023880084F8381084F83A30019200F00FFE019A70
:10239800A2858146E285E58DADB243464A462021B5
:1023A800204685B3E58DA768013DADB2B7F5805FDE
:1023B800E58512D0FFF714FF58BB236933B92368AA
:1023C8005B6833700136E6E70120CAE723685B687B
:1023D80003F07F0333700136DDE743464A46202188
:1023E8002046FFF7FDFEA0B9236933B923685B686F
:1023F800C3F3080326F8023BCDE723685B68DBB22A
:1024080026F8013BC7E784F83850284684F83A1084
:10241800A7E70320A5E700BF704700BF704700BFCC
:102428008368B3F5805F28D0036973B10368826A53
:102438005B68511C03F07F0381621370C38D013BFD
:102448009BB2C38543B100207047836A0268591C58
:10245800526881621A70F1E70268D16821F49071BC
:1024680010B5D1605169202421F00101516180F833
:102478003A40FFF7D3FF002010BD0269836A3AB9DA
:1024880002685268C2F3080223F8022B8362D5E778
:1024980002685268D2B223F8012B8362CEE700BFEC
:1024A800704700BF03681A6870B51607DD68596978
:1024B800044649D011F0010152D0D60705D5E805E8
:1024C80003D5E06B40F00100E06356077AD5002998
:1024D80000F08480E16B900741F00201E16376D55A
:1024E800E16B41F00401E163110772D4E16B00294B
:1024F80029D0910605D5AA0603D594F83A20222AB0
:102508007CD05D69E16B0E0702D415F040057AD0E6
:10251800DA6822F49072DA605A69202122F0010206
:102528005A6184F83A105A6955065ED55A69606B43
:1025380022F040025A61002857D03B4B036500F057
:1025480077FC002855D170BD96060CD5A9060AD58A
:1025580090F83A30222BF6D1BDE87040FFF760BF03
:1025680015F4907FA9D110060ED45606EBD56D064A
:10257800E9D5DA68202122F04002DA60204684F8A2
:102588003910FFF749FF70BD2906EED594F83920B8
:10259800212AD8D1A268B2F5805F226A38D0511CAE
:1025A800216212785A60E28C013A92B2E284002ADF
:1025B800C9D1DA6822F08002DA60DA6842F04002B3
:1025C800DA6070BD96070BD5002989D18EE711070F
:1025D8008CD5E16B41F00801E16387E7900785D46A
:1025E800100783D5002981D0F3E72046FFF758FF6D
:1025F80070BD606BBDE87040036D18472046FFF75B
:102608000FFF23687DE72046FFF74AFFE56370BDAB
:1026180011882069C1F30801596010B90232226299
:10262800C1E701322262BEE73526010808B5836B8F
:102638000022DA851846DA84FFF732FF08BD00BFAA
:10264800F0B50368DD0783B004462FD5A3498A682F
:1026580002F00C02042A00F0F4808A6802F00C02EE
:10266800082A00F0EA806368B3F5803F00F02C8107
:10267800B3F5A02F00F00081984D2A6822F480322B
:102688002A602A6822F480222A60002B40F0FD800C
:1026980000F08CFC064605E000F088FC801B6428EE
:1026A80000F2AA802B689B03F6D423689F072DD5D8
:1026B8008A4A916811F00C0F00F0A580916801F02A
:1026C8000C01082900F09B80E368002B00F0EB80E8
:1026D800834B824D01221A6000F068FC064605E033
:1026E80000F064FC801B022800F286802B689807A3
:1026F800F6D52968F82292FAA2F22369B2FA82F290
:1027080021F0F80193400B432B6023681A0720D46B
:10271800590734D4A369CBB1704DAA6802F00C02F2
:10272800082A77D0022B6F4B4FF000021A6000F096
:10273800D18000F03BFC2C46054604E000F036FC56
:10274800401B022858D823689B01F7D4002003B007
:10275800F0BD6369002B60D0634B604D01221A60A5
:1027680000F024FC064604E000F020FC801B022850
:1027780042D86B6F9F07F7D523685907CAD5574BBF
:102788005A4D002201921A6C42F080521A641B6C56
:1027980003F080530193019B2B6843F480732B60F3
:1027A80000F004FC064604E000F000FC801B022850
:1027B80022D82B68DA05F7D5A368012B00F0F18041
:1027C800052B00F0D580454D2A6F22F001022A67BB
:1027D8002A6F22F004022A67002B40F0D28000F012
:1027E800E5FB41F2883607462B6F980792D500F033
:1027F800DDFBC01BB042F7D9032003B0F0BD52681F
:1028080056023FF561AF354A1268950723D5E2684D
:10281800012A20D0012003B0F0BD334A2F4D1360A8
:1028280000F0C4FB064604E000F0C0FB801B022851
:10283800E2D86B6F9807F7D49EE74A6850027FF595
:1028480012AF264A126891037FF530AF6268002AFA
:102858007FF42CAFDEE7214DF821286891FAA1F129
:102868002269B1FA81F120F0F8008A4002432A6017
:102878001A077FF54DAF6CE7184B1A6842F48022AF
:102888001A601A6842F480321A6000F08FFB134D08
:10289800064604E000F08AFB801B6428ACD82B684D
:1028A8009A03F7D501E70E4A0C4D136000F07EFB42
:1028B800064604E000F07AFB801B02289CD82B68AF
:1028C8009907F7D4236821E7044A136843F480334F
:1028D8001360DAE700F06AFB06460FE000380240B2
:1028E8000000474260004742800E474200700040A7
:1028F80000F05CFB801B02283FF67EAF2B68990135
:10290800F6D447F6C07696FAA6F64FF44032B6FAF1
:1029180086F692FAA2F24FF07061B2FA82F091FA5A
:10292800A1F1A26A676AE369D4F820E0E46A520870
:1029380043EA0E0307FA06F6013A8240B1FA81F13A
:10294800334304FA01F11343194A1A4C0B4301218A
:102958006B60116000F02AFB054605E000F026FBDD
:10296800401B02283FF648AF23689A01F6D5EDE6EA
:10297800104B1A6F42F004021A671A6F42F00102F4
:102988001A6700F013FB0B4D074641F288362B6F90
:102998009B073FF5BFAE00F009FBC01BB042F6D95C
:1029A8002AE7044A136F43F001031367E9E700BFFE
:1029B8006000474200380240194A936803F00C034C
:1029C800042B2BD0082B27D15168536801F03F0105
:1029D80013F4800F536847F6C07292FAA2F0B0FA67
:1029E80080F003EA020323FA00F314BF0D480E48EF
:1029F800B0FBF1F000FB03F0094B4FF440325B6889
:102A080092FAA2F2B2FA82F203F44033D3400133CD
:102A18005B00B0FBF3F0704703487047014870470C
:102A28000038024040787D010024F400574A1368BA
:102A380003F00F038B4208D2CBB21370136803F074
:102A48000F03994201D00120704703689A072DE9C6
:102A5800F04106D54E4C8568A26822F0F0022A4360
:102A6800A260DF0706460C4626D54268012A00F018
:102A78008780931E012B464B1B687BD9990728D565
:102A8800434DAB6823F003031343AB6000F08EFAA9
:102A98007368012B074641F288384FD0022B58D073
:102AA800032B05D160E000F081FAC01B404564D8D3
:102AB800AB6813F00C0FF6D1344A136803F00F0318
:102AC8009C4209D2E3B21370136803F00F039C42CF
:102AD80002D00120BDE8F08133685A0706D52C4999
:102AE800F0688A6822F4E05202438A601B0707D51F
:102AF800274A3169936823F4604343EAC10393602A
:102B0800FFF75AFF224B0146F0229B6892FAA2F285
:102B1800B2FA82F203F0F003D3401E481E4AC35CA7
:102B2800002021FA03F3136000F008FA0020BDE842
:102B3800F08100F03BFAC01B40451ED8AB6803F09B
:102B48000C03042BF5D1B7E700F030FAC01B404561
:102B580013D8AB6803F00C03082BF5D1ACE700F0F1
:102B680025FAC01B404508D8AB6803F00C030C2BB2
:102B7800F5D1A1E7980183D4ABE70320BDE8F08144
:102B8800034B1B689D033FF57BAFA2E7003C024067
:102B9800003802409830010834000020084B4FF4F8
:102BA800E0529B6892FAA2F2B2FA82F203F4E0537E
:102BB800D3400449044ACB5C1068D840704700BF32
:102BC800003802409830010834000020084B4FF4C8
:102BD80060429B6892FAA2F2B2FA82F203F460436E
:102BE800D3400449044ACB5C1068D840704700BF02
:102BF8000038024098300108340000202DE9F04FD9
:102C0800D1F800C0DFF81482DFF814E283B00025A1
:102C180003E00135102D00F09B800123AB4003EA4F
:102C28000C029342F5D14E6826F0100ABAF1020F51
:102C380000F091804FEA45090324D0F800B004FA67
:102C480009F4E44306F003070BEA040B07FA09F753
:102C58000AF1FF3A47EA0B07BAF1010F076040F2A1
:102C6800A080C7688B683C4003FA09F32343C3601C
:102C7800F300CED54FF00009CDF80490D8F84430D1
:102C880043F48043C8F84430D8F8444025F003039F
:102C980003F1804304F4804403F59C33019405F068
:102CA8000304019FD3F808A0A4000F27A7402AEA2D
:102CB800070A544FB84222D007F58067B84200F09F
:102CC8008380514FB84200F08480504FB84200F0E2
:102CD80085804F4FB84200F086804E4FB84200F0D2
:102CE80087804D4FB84200F08880DFF8389148451A
:102CF8000CBF4FF007094FF0080909FA04F94AEA2E
:102D080009079F60DEF80030D443F70354BF23401F
:102D18001343CEF80030DEF80430B70354BF234025
:102D28001343CEF80430DEF80830F70254BF2340CE
:102D38001343CEF80830DEF80C30B60205F1010571
:102D480054BF23401343102DCEF80C307FF465AFE9
:102D580003B0BDE8F08F4FEAD50900EB890905F00B
:102D68000707D9F82040BF004FF00F0B0BFA07FBFD
:102D780024EA0B0A0C69BC4044EA0A04C9F820405A
:102D88004FEA45090324D0F800A004FA09F4E44303
:102D980006F003070AEA040A07FA09F747EA0A07E6
:102DA8000760876807EA040ACF6807FA09F747EA5D
:102DB8000A078760D0F804A0C6F300172AEA0303BD
:102DC800AF401F4347604CE74FF0010909FA04F987
:102DD80095E74FF0020909FA04F990E74FF0030963
:102DE80009FA04F98BE74FF0040909FA04F986E7B0
:102DF8004FF0050909FA04F981E74FF0060909FAC5
:102E080004F97CE70000024000080240000C024080
:102E1800001002400014024000180240003802402E
:102E2800003C0140001C024002B90904816170475E
:102E380090F83530022B03D080234365012070477A
:102E48000268052380F83530136823F00103136006
:102E580000207047074AD3684FF6FF010B40000275
:102E680043F0BF6300F4E06043F400330343D360EE
:102E7800704700BF00ED00E0184B70B4DC68C4F385
:102E88000224C4F10706042E04F1040328BF042613
:102E9800062B17D9033C0125A540013D2A400123F3
:102EA800B340013B1940A140002841EA02010CDB74
:102EB80000F1604000F561400901C9B280F80013D3
:102EC80070BC704700221446E9E7054B00F00F007C
:102ED80009010344C9B2197670BC704700ED00E0DF
:102EE800FCEC00E000F01F0101234009024A8B407E
:102EF80042F82030704700BF00E100E00138B0F12F
:102F0800807F0ED2084B10B4084C5860F02084F82B
:102F180023000022072110469A6019605DF8044BCF
:102F280070470120704700BF10E000E000ED00E0AE
:102F3800704700BF08B5FFF7FBFF08BD084B094AFB
:102F48001B6810B5A2FB032304469809FFF7D6FFB8
:102F5800214600224FF0FF30FFF78EFF002010BD02
:102F680034000020D34D621008B50B4B1A6842F4A8
:102F780000721A601A6842F480621A601A6842F491
:102F880080721A600320FFF765FF0020FFF7D6FF65
:102F9800FEF7DEFB002008BD003C0240024A136831
:102FA80001331360704700BFB8010020014B186857
:102FB800704700BFB801002010B582B00190FFF73C
:102FC800F5FF0446FFF7F2FF019B001B9842F9D377
:102FD80002B010BD1049114BD1F8882042F470029C
:102FE80010B4C1F888201A680D4C002042F0010284
:102FF8001A6098601A6822F0847222F480321A608B
:103008005C601A684FF0006422F480221A60D8606D
:103018008C605DF8044B704700ED00E0003802401A
:1030280010300024DFF834D0002103E00C4B5B584B
:10303800435004310B480C4B42189A42F6D30B4AC2
:1030480002E0002342F8043B094B9A42F9D3FFF708
:10305800C1FFFDF7E7F8FEF7ABF870470000022064
:10306800B03001080000002038000020380000209F
:10307800BC010020FEE70000F8B500BFF8BC08BCA2
:103088009E467047F8B500BFF8BC08BC9E4670471E
:1030980000000000010203040102030406070809F6
:0430A800F501010825
:0430AC00CD01010849
:1030B000B6000000FF000000FF00000000000D004F
:1030C000FE00010001000000FE00020002000000FE
:1030D000636F6E6E656374006E6F7420636F6E6EE7
:0830E000656374000024F40094
:040000050801302D91
:00000001FF
